:100000000C9411040C9455040C9455040C94550450
:100010000C9455040C9455040C9455040C945504FC
:100020000C9455040C9455040C94FE0F0C94D010B1
:100030000C9455040C9455040C9455040C945504DC
:100040000C9455040C94DA240C9455040C94550427
:100050000C9455040C946D1E0C9455040C9455048A
:100060000C9455040C9455040C9455040C945504AC
:100070000C9455040C9455040C9455040C9455049C
:100080000C9455040C9455040C9455040C9455048C
:100090000C9455040C9455040C9455040C9455047C
:1000A0000C9455040C9455040C9455046907D4061B
:1000B0008007220733075107EC0616071C071007B5
:1000C0004B0727072D0704070A07BA063D115F11E2
:1000D0004D125F114D12A411C7114D121C122F1297
:1000E000FE14FE142D152D1563158315B416B416C4
:1000F0008E15B4163E163E16A516B416B416AE16D8
:100100004B164B164B164B164B164B164B164B16E7
:100110004B164B164B164B164B164B164B164B16D7
:100120005D166A1671167816821602E002E2012E3A
:10013000022E02E10002E002E102E20001E001E140
:1001400001E20002E001E30119021902E30002E00A
:100150000001E00002E002E3016402640002E00248
:10016000E30001E001E30001E10137023702E101B0
:1001700038023801E10125022502E10002E002E136
:10018000013102310002E002E10001E001E1000181
:10019000E10137023702E10138023801E1010702CB
:1001A0000702E10001350235012002200002E302CE
:1001B000E10001E301E10001E10136023602E10163
:1001C00038023801E10126022602E10001E101378F
:1001D000023702E10138023801E10126022602E17C
:1001E0000001E10136023602E10138023801E10185
:1001F00025022502E10001E10137023702E1013861
:10020000023801E20125022502E20001E101370284
:100210003702E10138023801E10130023002E10029
:1002200002E002E2013002300002E002E20001E0FE
:1002300001E20002E001E30106020602E30002E03F
:100240000001E00029002B00E200E1003541000040
:100250001E00140004001D7105304D431F001A00DC
:1002600016001B0006304C002000080007000600A6
:1002700052002A00210015000900190051004A000F
:10028000220017000A000500000002300430E300DD
:100290000000E200000002540430E7000000E60025
:1002A0000000045423001C000B00110000002E7FEE
:1002B000240018000D00100050004B0025000C0019
:1002C0000E0036004F002C00260012000F003700F1
:1002D000E10828002700130033003871E1044E00C4
:1002E0002D002F003474E5003041000001000100B2
:1002F00001000100010000003A003500310001005A
:10030000010001003B0035022102350001004C00D4
:100310003C001E0224062202010001003D002D02C5
:1003200024022404010001003E00010037001104F2
:1003300000000100010001000000010000000100B8
:100340000F30010000000100000068003F0024069B
:100350002402240400004500400022042502110468
:1003600031026900410023042602640050000100AC
:1003700042003500250452005100010043003502BF
:10038000260438004F006A0044001E02310021029A
:100390000100000001000100010001000100000057
:1003A0000100010001000100010001000100F40052
:1003B000F200FB00010001000100F000F100FA0072
:1003C000010001000100F500F300FC000100010044
:1003D0000100F900FA00F600000001000100010030
:1003E0000000010000000100A80001000000010061
:1003F0000000010001000100A900AA0000000100A6
:1004000001000100010001000100010001000100E4
:100410000100AC000100B600010001000100AB00CA
:1004200050000100010001000100520051000100D4
:10043000AE000100010001004F00000001000100BA
:1004400001000100010000000100010001000100A5
:100450000100010001000100010001000100010094
:100460000100010001000100010001000100010084
:100470000100010001000100010001000100010074
:100480000000010001000100000001000000010067
:1004900007300100000001000000010008300E30AC
:1004A0000B300100000001000C300A300D3001005B
:1004B00001000100010009300100010001000100FC
:1004C0000100010001000100010001000100010024
:1004D0000100010001000100010001000100010014
:1004E0000100000001000100010001000100000006
:1004F00001000100010001000100010001000100F4
:1005000050000100010001000100520051000100F3
:1005100001000100010001004F0001000100010085
:1005200001000100010001000000010001000100C4
:1005300000000100000001000100010000000100B6
:10054000000001003F0052005100230200000100A2
:100550004000240021001E0027000100410025006A
:1005600022001F0037000100420026002300200067
:10057000360001004300300230002402270201004F
:1005800044004500380001000100000001000100A6
:10059000E1000100E0000000010001000100010095
:1005A00001003D0001000100010001000100E00028
:1005B000010001000100010001002C000100010008
:1005C0000100010001003C000100010001000100E8
:1005D00000003A00010001000000010000003B00A3
:1005E0000F300100000001000000010001000100C7
:1005F00001000100000001000100010001000100F4
:1006000001000100010001000100010001000100E2
:1006100001000100010001000100010001000100D2
:1006200001000100010001000100010001000100C2
:100630000100000016034500720067006F004400CF
:100640006F007800200045005A00000016034500A6
:10065000720067006F0044006F00780020004500C2
:100660005A0000000403090409026D00040100A0FF
:10067000FA09040000010301010009211101000130
:10068000223F000705810308000A09040100010355
:10069000010200092111010001224D00070582031A
:1006A00008000A09040200010300000009211101E9
:1006B00000012236000705830308000A090403002D
:1006C0000103000000092111010001223900070582
:1006D00084031000011201100100000008EDFE0764
:1006E0001301000102000105010906A10105071916
:1006F000E029E71500250195087501810205081913
:100700000129059505750191029501750391010572
:10071000071900297715002501957875018102C018
:1007200005010980A101850216010026B7001A0102
:10073000002AB700751095018100C0050C0901A1C0
:10074000018503160100269C021A01002A9C0275ED
:100750001095018100C005010902A1010901A10054
:100760000509190129051500250195057501810265
:100770009501750381010501093009311581257F36
:1007800095027508810609381581257F9501750840
:100790008106050C0A38021581257F9501750881AF
:1007A00006C0C005010906A101050719E029E715E2
:1007B00000250195087501810295017508810105E3
:1007C0000819012905950575019102950175039197
:1007D000010507190029FF150025FF9506750881F9
:1007E00000C0000000000000000000000001020442
:1007F000060A0F17202C3A4A5D71879DB3C7DAE9C4
:10080000F5FCFFFCF5E9DAC7B39D87715D4A3A2C28
:1008100020170F0A0604020100000000000000007B
:10082000000011241FBECFEFDAE0DEBFCDBF04B65B
:1008300003FE24C08091FD019091FE01A091FF0173
:10084000B09100028730904BA740B04BB9F41092A2
:10085000FD011092FE011092FF011092000214BEE1
:1008600084B7877F84BF88E10FB6F89480936000D7
:10087000109260000FBEE0E0FFE3099511E0A0E0F8
:10088000B1E0E2E4FDE402C005900D92A433B107AB
:10089000D9F711E0A4E3B1E001C01D92AD3FB1076B
:1008A000E1F70E94420D0C949F260C9400001092D8
:1008B000B9008AE08093B800089594EA9093BC0050
:1008C0009091BC0097FFFCCF9091B900987F983031
:1008D00021F0903111F081E008958093BB0084E80D
:1008E0008093BC008091BC0087FFFCCF8091B90051
:1008F000887F883111F0803471F780E0089584E9B1
:100900008093BC008091BC0084FDFCCF089580934F
:10091000BB0084E88093BC008091BC0087FFFCCFC3
:100920009091B900987F81E0983209F480E00895B1
:1009300084E88093BC008091BC0087FFFCCF80914D
:10094000BB00089580910101811115C080E40E94CF
:100950005D048093010181110CC082E10E94870433
:1009600080930101811105C08FEF0E94870480935D
:1009700001010E947F0484B1807F84B985B1807FAA
:1009800085B98AB1837F8AB98BB1837F8BB93E9851
:10099000469808950E945D06809301010E94A2047A
:1009A00080B38C7080BB81B3836F81BBA5E3B1E062
:1009B000E3E4F1E08EE08E0F11921D928E13FCCFD6
:1009C0000C944706BF92CF92DF92EF92FF920F9363
:1009D0001F93CF93DF9380910101882379F0809159
:1009E00034018F5F80933401811108C00E945D063D
:1009F00080930101811102C00E94EF0505E311E01F
:100A0000C0E0D0E0DD24D39482E0C82EEE24E3944D
:100A1000F12CC730D10500F580910101811164C02E
:100A200080E40E945D0480930101811112C082E183
:100A30000E9487048093010181110BC0C7010C2E15
:100A400001C0880F0A94EAF780950E94870480937A
:100A500001010E947F0448C0CA30A1F028F4C830C8
:100A600059F0C93061F005C0CC3089F070F0CD305C
:100A700089F0209A289810C0219A29980DC0229AAE
:100A80002A980AC0239A2B9807C0529A01C0539AF9
:100A90005B9802C03E9A469890EA9A95F1F79FB10A
:100AA000799902C082E001C080E091709D25982B69
:100AB0007C9902C084E001C080E0892B7D9902C04E
:100AC00038E001C030E0832B7E9902C020E101C0F4
:100AD00020E0822B9FB19095991F9927991F92959D
:100AE000990F907E892B0FC080910101811149C01F
:100AF00080E40E945D0480930101882379F1B12C88
:100B00000E947F048B2DF8019081981719F0808343
:100B1000C09200010E94A20421960F5F1F4FCE30A9
:100B2000D10509F076CF80910001882361F18150D1
:100B300080930001882339F08FE99FE00197F1F756
:100B400000C0000020C0A3E4B1E0E5E3F1E0CF0184
:100B5000825F91919D938E13FCCF15C083E10E941B
:100B60008704809301018111CACF81E40E945D0452
:100B7000809301018111C3CF0E949804B82EB094D4
:100B8000BFCF80E0C0CF0E94ED0581E0DF91CF9123
:100B90001F910F91FF90EF90DF90CF90BF9008953D
:100BA000E82FF0E0ED5BFE4F8081089508950F93EC
:100BB0001F93CF93DF93C3E4D1E010E00C2F025FCB
:100BC000899190E00E94931D180F0C13F9CF812F8B
:100BD000DF91CF911F910F9108950C94B007569813
:100BE0005E9825982D9826982E9827982F988FEF05
:100BF00090E0909389008093880090938B0080937D
:100C00008A0090938D0080938C00259A2D9A2FEF67
:100C100080E792E0215080409040E1F700C0000062
:100C2000269A2E9A2FEF80E792E021508040904044
:100C3000E1F700C00000279A2F9A2FEF80E792E09B
:100C4000215080409040E1F700C0000025982D9889
:100C50002FEF80E792E0215080409040E1F700C004
:100C6000000026982E982FEF80E792E021508040D8
:100C70009040E1F700C0000027982F9856985E98A2
:100C800025982D9826982E9827982F98089589EAC8
:100C90008093800089E08093810024982C983F986D
:100CA0008AB18F748AB96E98479A8BB1806B8BB971
:100CB000769A0E94EF050C94AF0780E280930101C1
:100CC0008091510181110EC00E94570481E08093F0
:100CD00051012FEF83ED90E3215080409040E1F7E8
:100CE00000C0000080E40E945D0480930101811136
:100CF0002EC00E94870480930101811128C00E94A8
:100D0000870480930101811122C08FE30E94870430
:100D10008093010181111BC00E947F0480E40E9426
:100D20005D0480930101811112C08CE00E94870450
:100D30008093010181110BC00E94870480930101FF
:100D4000811105C08FE30E948704809301010E94F6
:100D50007F04809101010895462F50E040315105F4
:100D600008F0F1C0DC01FA01EA5AFF4F12968C91AB
:100D70000C944F26882309F4E6C08091BF0190911E
:100D8000C001A091C101B091C20120E2822780720E
:100D90009927AA27BB278093BF019093C001A093F6
:100DA000C101B093C201CFC0882349F00E94371E11
:100DB000909353018093520181E492E008958091D1
:100DC0005201909153010E94431E873991050CF006
:100DD000AEC083E392E00895882349F00E94371E55
:100DE00090935301809352018EE292E00895809196
:100DF0005201909153010E94431E873991050CF0D6
:100E000099C080E292E00895882309F49CC08BE0A9
:100E100092E00895882309F496C086EF91E0089542
:100E2000882309F490C081EE91E00895882309F4A5
:100E30008AC08CEC91E00895882309F484C087EB84
:100E400091E00895811179C08DEA91E00895882399
:100E500009F479C084EA91E00895882309F473C005
:100E60008FE891E00895882349F00E94371E9093FF
:100E70005301809352018AE891E0089580915201D4
:100E8000909153010E94431E873991050CF058C080
:100E90008CE791E00895882309F455C087E691E036
:100EA0000895882349F00E94371E90935301809340
:100EB000520182E691E00895809152019091530190
:100EC0000E94431E873991050CF040C084E591E0F3
:100ED0000895882349F00E94371E90935301809310
:100EE000520181E591E00895809152019091530162
:100EF0000E94431E8739910564F583E491E00895CB
:100F0000882349F00E94371E909353018093520129
:100F10008CE391E0089580915201909153010E94D9
:100F2000431E87399105C4F48AE291E008958EE367
:100F300092E0089589E292E0089582EB91E00895AD
:100F400085E891E0089580E090E008958DE591E0D6
:100F500008958EE491E0089585E391E00895089561
:100F60006091BF017091C0018091C1019091C20157
:100F70000E949F1D56985E9825982D9826982E9829
:100F800027982F988330C1F028F4813041F08230C7
:100F900049F00895843049F0853051F00895259A3C
:100FA0002D9A0895269A2E9A0895259A2D9A04C06E
:100FB000259A2D9A269A2E9A279A2F9A089581E09B
:100FC000089581E008950C94E10708950F931F930D
:100FD000CF93DF938C01FC01C081D181CE010E94AF
:100FE000181CBE010E948F08EC01B8010E94E307A3
:100FF000882309F48DC0F8018281882309F44AC04E
:1010000080915F0181111FC0C431F0E5DF0709F055
:1010100051C00E94E50781E080935F010E94371E66
:1010200090935E0180935D011092560110925801D9
:101030001092570110925A011092590110925C01BE
:1010400010925B0165C080915D0190915E010E94EC
:10105000431E883C910570F480915601E82FF0E022
:10106000EE0FFF1FE95AFE4FD183C0838F5F80933D
:1010700056014EC0C43880E5D80721F0C538D045A8
:1010800001F13AC0F8018281882341F010925401A5
:1010900082E01EC0C438E0E5DE0759F580915401B6
:1010A000811106C086E20E94A21386E20E946A14A1
:1010B00082E01CC0C438F0E5DF0741F3C538D045F5
:1010C000D9F4F8018281882331F01092550180E231
:1010D0000E94B9141DC080915501811106C087E29C
:1010E0000E94A21387E20E946A1480E20E94C01448
:1010F0000FC0C538D04529F381E080935401809317
:101100005501C801DF91CF911F910F910C94DF071A
:1011100080E0DF91CF911F910F910895089596E09F
:10112000799FF001112494E5899FE00DF11D1124B0
:10113000E60FF11DEE0FFF1FEC5BFD4F85919491C3
:101140000895880F991FFC01EC53FF4F85919491EE
:101150000895880F991FFC01EC5BFD4F85919491D8
:1011600008950F931F93CF93DF93EC01811520E334
:10117000920750F5C11580E2D80708F0C3C0CB3BF9
:10118000D10590F4C83AD10508F06AC0C53AD10536
:1011900008F05BC0C430D10508F0D0C1219709F038
:1011A000CAC101E010E00AC2CF3FD10511F008F03A
:1011B000C5C1C03FD10508F0A2C0CE01805E910933
:1011C000089708F4BBC1B7C1C13090E5D90709F44D
:1011D000A2C020F5C0318FE4D80770F4C11590E4A7
:1011E000D90708F094C0C11521E3D20708F0A3C1C4
:1011F000DD278E01106CE2C1C115D04509F09BC1FD
:101200000E941F178FEF94E32CE081509040204004
:10121000E1F700C000000E94921ED0C1C11597E501
:10122000D90758F4C03121E5D20708F01CC1C431F8
:1012300080E5D80708F475C07EC1CE0190578115AE
:10124000904108F078C1DF7073C1C53AD10509F447
:1012500077C1C63AD10509F076C102E810E4AEC103
:10126000C83AD10509F472C1C93AD10509F471C16E
:10127000CA3AD10509F470C1CB3AD10509F46FC15E
:10128000CC3AD10509F46EC1CD3AD10509F46DC14E
:10129000C03BD10509F46CC1CE3AD10509F46BC14C
:1012A000CF3AD10509F46AC1C13BD10509F469C13E
:1012B000C23BD10509F468C1C33BD10509F467C13C
:1012C000C43BD10509F466C1C53BD10509F465C12C
:1012D000C63BD10509F464C1C73BD10509F463C11C
:1012E000C83BD10509F462C1C93BD10509F461C10C
:1012F000CA3BD10509F460C100E014E45FC18E016E
:1013000010655CC1CE019F700E94A90858C1DF70B2
:101310008E01106A53C18091DC0181608093DC01F1
:101320004DC10E943720811102C00E941D200E94E1
:10133000542090E09093FD018093FC01C23080E541
:10134000D80721F48091FC01816086C0C43090E50B
:10135000D90721F48091FC0182607EC0C63020E56F
:10136000D20721F48091FC01846076C0C83080E50A
:10137000D80719F48091FC0127C0CA3090E5D9073D
:1013800021F48091FC01806167C0CC3020E5D20758
:1013900021F48091FC0180625FC0CE3080E5D807E7
:1013A00021F48091FC01806457C0C03190E5D907D9
:1013B00021F48091FC0180684FC0C23120E5D20742
:1013C00029F48091FC018460886046C0C33080E5C8
:1013D000D80721F48091FC018E7F3EC0C53090E596
:1013E000D90721F48091FC018D7F36C0C73020E5FC
:1013F000D20721F48091FC018B7F2EC0C93080E59B
:10140000D80719F48091FC0126C0CB3090E5D907AC
:1014100021F48091FC018F7E1FC0CD3020E5D207E2
:1014200021F48091FC018F7D17C0CF3080E5D80773
:1014300021F48091FC018F7B0FC0C13190E5D90769
:1014400021F48091FC018F7707C0C331D04531F47E
:101450008091FC018B7F877F8093FC018091FC0150
:101460000E945820ABC08D2F99278F70992781300B
:101470009105D9F49E012370332702C0880F991F6C
:101480002A95E2F79C688E0144E0000F111F4A95EF
:10149000E1F700271370802B912B53E0CC0FDD1F59
:1014A0005A95E1F7C076DD272FC08230910531F4DF
:1014B000DC2FCC278E01016F106A80C0833091052C
:1014C00069F4CE018370992701E010E002C0000F9B
:1014D000111F8A95E2F7C8019C680FC084309105FE
:1014E000B9F4CE018370992701E010E002C0000F2B
:1014F000111F8A95E2F7C8019A6823E0CC0FDD1F1F
:101500002A95E1F7C07ED7708C010C2B1D2B56C09D
:101510008530910531F4DC2FCC278E01046F106AE1
:101520004DC0069709F04AC0CF71DD27DC2FCC27CC
:101530008E01106243C000E010E040C08E013EC04A
:1015400001E810E43BC003E810E438C002EE14E404
:1015500035C009EE14E432C00AEE14E42FC005EBE6
:1015600014E42CC006EB14E429C007EB14E426C0F5
:101570000CEC14E423C00DEC14E420C003E815E4E3
:101580001DC00AE815E41AC002E915E417C004E911
:1015900015E414C001E216E411C003E216E40EC023
:1015A00004E216E40BC005E216E408C006E216E405
:1015B00005C007E216E402C00AE216E4C801DF91A2
:1015C000CF911F910F91089596E0799FF00111241A
:1015D00094E5899FE00DF11D1124E60FF11DEE0F3A
:1015E000FF1FEC5BFD4F85919491803E9105E0F4E7
:1015F000803C910558F58133910509F46FC048F49A
:101600008932910509F463C08A32910509F46DC0ED
:1016100072C089339105E9F082389105D1F08533A4
:10162000910509F44DC067C0833E910581F138F4FE
:10163000803E9105B9F0823E9105D9F05CC0863EAE
:10164000910561F1873E9105A1F155C00E94A10865
:1016500008952091FC0120FD02C021FF4CC080EEC6
:1016600090E049C08091FC0180FFF9CF89E390E0D0
:1016700042C08091FC0182FF0EC08091FC0184FF7A
:1016800003C080E090E037C083EE90E034C08091EA
:10169000FC0182FFF2CF82EE90E02DC08091FC0130
:1016A00083FF0BC08091FC0184FDEBCF87EE90E0BF
:1016B00022C08091FC0183FFF5CF86EE90E01BC035
:1016C0008091FC0185FF07C089E290E014C0809101
:1016D000FC0185FFF9CF85E390E00DC08091FC010E
:1016E00086FF07C08AE290E006C08091FC0186FF79
:1016F000F9CF81E390E00E94B108089508950C9419
:101700007E0B809170010895CF93DF9300D01F92DC
:10171000CDB7DEB79C018091F301843019F593E0D9
:1017200099833B832A839093E9008FEF9091E8009F
:10173000815095FD06C095ED9A95F1F70000811155
:10174000F5CF8091E80085FF0DC040E050E063E0F8
:1017500070E0CE0101960E94EE0D8091E8008E7738
:101760008093E8000F900F900F90DF91CF91089534
:10177000CF93DF9300D01F92CDB7DEB72091F30156
:10178000243021F522E029839B838A8383E08093A0
:10179000E9008FEF9091E800815095FD06C095ED2E
:1017A0009A95F1F700008111F5CF8091E80085FF4F
:1017B0000DC040E050E063E070E0CE0101960E9471
:1017C000EE0D8091E8008E778093E8000F900F90E7
:1017D0000F90DF91CF9108952091F3012430F1F41F
:1017E00022E02093E9002FEF3091E800215035FDF1
:1017F00006C035ED3A95F1F700002111F5CF2091A3
:10180000E80025FF0BC040E050E065E070E00E947A
:10181000EE0D8091E8008E778093E8000895CF93D5
:10182000DF93EC019091F301943009F046C0809170
:101830000C018823D9F080910D018823B9F0909391
:10184000E9008FEF9091E800815095FD06C095E189
:101850009A95F1F700008111F5CF8091E80085FF9E
:101860002CC040E050E060E170E017C081E0809360
:10187000E9008FEF9091E800815095FD06C095ED4D
:101880009A95F1F700008111F5CF8091E80085FF6E
:1018900014C040E050E068E070E0CE010E94EE0D20
:1018A0008091E8008E778093E80080E1FE01A0E659
:1018B000B1E001900D928A95E1F7DF91CF91089503
:1018C0008091F201811109C00E94830F0E94E00FF4
:1018D0008091E20084608093E20008951092F2010A
:1018E000089508950C94C7240E94281E0E94CD24B8
:1018F0000E9486120C947F0B42E061EC81E00E9412
:10190000FD0E42E061EC82E00E94FD0E42E061ECDF
:1019100083E00E94FD0E42E161EC84E00C94FD0E38
:101920008091F501833009F455C030F4813071F0B5
:10193000823009F48EC008958A3009F47AC08B3061
:1019400009F460C0893009F09CC020C08091F40186
:10195000813A09F096C08091E800877F8093E80083
:101960008091F8019091F901892B21F460E180E6E2
:1019700091E003C060E080E090E070E00E94390EEA
:101980008091E8008B778093E80008958091F401BE
:10199000813209F076C08091F8019091F9010097A9
:1019A00019F0039709F06DC08091E800877F80935C
:1019B000E8008091E80082FD05C08091F30181116B
:1019C000F8CF5FC08091F100809370018091E800B2
:1019D0008B7753C08091F401813A09F052C0809115
:1019E000F8019091F901892B09F04BC08091E80032
:1019F000877F8093E8008091E80080FFFCCF809192
:101A00000C0136C08091F4018132D9F58091F80142
:101A10009091F901892BA9F58091E800877F809347
:101A2000E8000E94320F8091F60180930C010C9423
:101A30001F178091F401813221F58091E800877FA2
:101A40008093E8000E94320F8091F701809371012A
:101A500008958091F401813AA1F48091E800877F94
:101A60008093E8008091E80080FFFCCF80917101B5
:101A70008093F1008091E8008E778093E8000C94C9
:101A8000320F089584B7877F84BF88E10FB6F8943A
:101A900080936000109260000FBE90E080E80FB667
:101AA000F89480936100909361000FBE0E94D5125C
:101AB0000E94830F0E94E00F8091E2008460809377
:101AC000E20078940E9466120E94D71282E091E0B0
:101AD0000E9481120E94B5248091F301853069F43F
:101AE0000E94EF1D8091F1018823B1F30E941A1E1C
:101AF000882391F30E94D80DEFCF0E94DD12ECCF26
:101B0000292F332723303105C9F064F42130310502
:101B100081F02230310509F043C08DE690E028E6DF
:101B200036E042C021323105F1F02232310541F177
:101B300037C082E190E025ED36E036C0992781304C
:101B4000910541F08230910541F0892B49F5E4E699
:101B5000F6E005C0ECE4F6E002C0E4E3F6E08491D0
:101B600090E09F0121C06430D8F4E62FF0E0EE0F42
:101B7000FF1FEE5DFE4F2081318189E090E014C0AF
:101B8000643070F470E0FB01EE0FFF1FE65EFE4F65
:101B900020813181FB01EA5EFE4F808190E004C02C
:101BA00080E090E020E030E0FA0131832083089566
:101BB00080E189BD82E189BD09B400FEFDCF80913D
:101BC000D8008F7D8093D8008091E0008260809360
:101BD000E0008091E00081FDFCCF0895CF92DF927C
:101BE000EF92FF920F931F93CF93DF93EC018B0142
:101BF0006A010E94510F811133C0C114D10439F020
:101C0000F60180819181081B190BC80FD91FE12CA7
:101C1000F12C0115110519F18091E80085FD16C020
:101C20008091E8008E778093E800C114D10449F0D8
:101C3000F60180819181E80EF91EF182E08285E053
:101C40000FC00E94510F882321F30AC0899180930D
:101C5000F10001501109FFEFEF1AFF0ADACF80E01F
:101C6000DF91CF911F910F91FF90EF90DF90CF9078
:101C700008952091FA013091FB012617370748F0AB
:101C80006115710539F42091E8002E772093E80062
:101C900001C0B90140E061157105A9F12091F3017E
:101CA000222309F443C0253009F442C02091E80002
:101CB00023FD40C02091E80022FD32C02091E800C1
:101CC00020FFE9CF4091F3002091F20030E0342B67
:101CD000FC01CF016115710559F02830310540F440
:101CE00081918093F100615071092F5F3F4FF1CFD7
:101CF00041E02830310509F040E02091E8002E77DE
:101D00002093E800C8CF4111C9CF0AC08091F301E8
:101D1000882361F0853061F08091E80083FD0AC07E
:101D20008091E80082FFF2CF80E0089582E008957C
:101D300083E0089581E008952091FA013091FB013C
:101D40002617370748F06115710539F42091E8002E
:101D50002E772093E80001C0B901FC0120E0611555
:101D6000710591F18091F301882309F440C0853019
:101D700009F43FC08091E80083FD3DC08091E800F8
:101D800082FD2FC08091E80080FFE9CF2091F30011
:101D90008091F20090E0922B6115710559F0883026
:101DA000910540F424912093F1003196615071091E
:101DB0000196F2CF21E0089709F020E08091E80039
:101DC0008E778093E800CBCF2111CCCF0AC08091D1
:101DD000F301882361F0853061F08091E80083FD94
:101DE0000AC08091E80082FFF2CF80E0089582E08F
:101DF000089583E0089581E00895982F973058F56D
:101E00009093E900981739F07091EC002091ED0063
:101E10005091F00003C0242F762F50E021FF19C00D
:101E20003091EB003E7F3093EB003091ED003D7F31
:101E30003093ED003091EB0031603093EB00709304
:101E4000EC002093ED005093F0002091EE0027FF6E
:101E500007C09F5FD3CF8F708093E90081E0089522
:101E600080E008958091F40187FF11C08091E8001F
:101E700082FD05C08091F3018111F8CF11C08091DE
:101E8000E8008B770BC08091F301882349F08091A3
:101E9000E80080FFF8CF8091E8008E778093E8001B
:101EA00008952091E4003091E50095E64091EC0022
:101EB000842F817040FF22C08091E80080FD1CC00B
:101EC0008091F301882391F0853091F08091EB00AF
:101ED00085FD10C04091E4005091E5004217530782
:101EE00029F39A01915011F784E0089582E0089552
:101EF00083E0089581E0089580E008954091E8002E
:101F000042FFDECF08950E94F10F0E94F90FE0EE2C
:101F1000F0E0808181608083E8EDF0E080818F7760
:101F2000808319BCA7EDB0E08C918E7F8C9380816B
:101F30008F7E80831092F20108950F931F93CF93A9
:101F4000DF930E94F10F0E94F90FC8EDD0E0888165
:101F50008F77888388818068888388818F7D888354
:101F600019BC1092F3011092EF011092F10110923E
:101F7000F00100EE10E0F80180818B7F8083888182
:101F80008160888342E060E080E00E94FD0EE1EE27
:101F9000F0E080818E7F8083E2EEF0E080818160DE
:101FA0008083808188608083F80180818E7F808338
:101FB000888180618883DF91CF911F910F9108956F
:101FC000E8EDF0E080818F7E8083E7EDF0E08081B6
:101FD0008160808384E082BF81E08093F2010C9471
:101FE0009D0FE8EDF0E080818E7F80831092E2000B
:101FF00008951092DA001092E10008951F920F9256
:102000000FB60F9211242F933F934F935F936F93CB
:102010007F938F939F93AF93BF93EF93FF938091A1
:10202000E10082FF0BC08091E20082FF07C0809137
:10203000E1008B7F8093E1000E9465128091DA00BD
:1020400080FF1FC08091D80080FF1BC08091DA0004
:102050008E7F8093DA008091D90080FF0DC080E1EF
:1020600089BD82E189BD09B400FEFDCF81E0809386
:10207000F3010E94600C05C019BC1092F3010E948C
:102080006E0C8091E10080FF19C08091E20080FF1A
:1020900015C08091E2008E7F8093E2008091E20083
:1020A00080618093E2008091D80080628093D800A4
:1020B00019BC85E08093F3010E94720C8091E100CD
:1020C00084FF30C08091E20084FF2CC080E189BD94
:1020D00082E189BD09B400FEFDCF8091D8008F7DDB
:1020E0008093D8008091E1008F7E8093E100809101
:1020F000E2008F7E8093E2008091E2008160809315
:10210000E2008091EF01882311F084E007C0809104
:10211000E30087FD02C081E001C083E08093F3010A
:102120000E94740C8091E10083FF29C08091E2003D
:1021300083FF25C08091E100877F8093E10082E0EA
:102140008093F3011092EF018091E1008E7F8093E4
:10215000E1008091E2008E7F8093E2008091E200B6
:1021600080618093E20042E060E080E00E94FD0E2A
:102170008091F00088608093F0000E94710CFF91C4
:10218000EF91BF91AF919F918F917F916F915F91EF
:102190004F913F912F910F900FBE0F901F90189568
:1021A0001F920F920FB60F9211242F933F934F93CC
:1021B0005F936F937F938F939F93AF93BF93CF93CF
:1021C000DF93EF93FF93C091E900CF708091EC0013
:1021D000D82FD17080FDD0E81092E9008091F000F6
:1021E000877F8093F00078940E9414111092E90088
:1021F0008091F00088608093F000CD2BCF70C09369
:10220000E900FF91EF91DF91CF91BF91AF919F9145
:102210008F917F916F915F914F913F912F910F908F
:102220000FBE0F901F9018951F93CF93DF93CDB7DC
:10223000DEB7AA970FB6F894DEBF0FBECDBFE4EFAE
:10224000F1E088E08E0F9091F10091938E13FBCF17
:102250000E94900C8091E80083FF1FC18091F401DF
:102260009091F501492F50E04A30510508F015C111
:10227000FA01EA59FF4F0C944F26803881F08238DA
:1022800009F00BC18091F8018F708093E900809173
:10229000EB0085FB882780F91092E90006C0809149
:1022A000F0019091F101911182609091E800977F87
:1022B0009093E8008093F1001092F100C8C0282F9D
:1022C0002D7F09F0EAC0882319F0823061F0E5C063
:1022D0008091F601813009F0E0C0933009F080E090
:1022E0008093F1012BC08091F601811127C080916C
:1022F000F8018F7009F4D1C08093E9002091EB00C0
:1023000020FF1CC0933021F48091EB00806214C048
:102310009091EB0090619093EB0021E030E0A901F7
:1023200002C0440F551F8A95E2F74093EA001092CD
:10233000EA008091EB0088608093EB001092E90046
:102340008091E800877F86C08111A7C01091F601B7
:102350001F778091E3008078812B8093E300809148
:10236000E800877F8093E8000E94320F8091E800A8
:1023700080FFFCCF8091E30080688093E30011111F
:1023800002C082E001C083E08093F30186C08058E0
:10239000823008F082C08091F6019091F7018C3D67
:1023A00053E0950779F583E08A838AE289834FB702
:1023B000F894DE01139620E03EE051E2E32FF0E0D6
:1023C00050935700E49120FF03C0E295EF703F5F08
:1023D000EF708E2F90E0EA3010F0C79601C0C096E3
:1023E0008D939D932F5F243149F74FBF8091E80073
:1023F000877F8093E8006AE270E0CE0101960E9438
:10240000390E14C0AE014F5F5F4F6091F8010E941A
:10241000800DBC01009709F440C09091E800977FBF
:102420009093E80089819A810E949C0E8091E80037
:102430008B778093E80031C0803879F58091E8008F
:10244000877F8093E8008091EF018093F100809175
:10245000E8008E778093E8000E94320F1EC0811141
:102460001CC09091F6019230C0F48091E800877F03
:102470008093E8009093EF010E94320F8091EF016A
:10248000811106C08091E30087FD02C081E001C098
:1024900084E08093F3010E947C0C8091E80083FF2C
:1024A0000AC08091E800877F8093E8008091EB006C
:1024B00080628093EB00AA960FB6F894DEBF0FBE41
:1024C000CDBFDF91CF911F9108950895CF93809153
:1024D000F3018823A1F0C091E900CF709091EC0046
:1024E000892F817090FD80E8C82B1092E9008091BF
:1024F000E80083FD0E941411CF70C093E900CF91D2
:10250000089590937701809376010895E091760184
:10251000F0917701309721F00190F081E02D09943E
:1025200080E00895E0917601F0917701309721F0F5
:102530000280F381E02D09940895E0917601F091F5
:102540007701309721F00480F581E02D09940895FA
:1025500020917401309175018217930771F0909367
:10256000750180937401E0917601F09177013097C5
:1025700021F00680F781E02D0994089520917201E1
:10258000309173018217930771F0909373018093D8
:102590007201E0917601F0917701309721F000848B
:1025A000F185E02D0994089508950C94D4120E94A9
:1025B0002E1E0E94CA040C94F01E9F92AF92BF92EE
:1025C000CF92DF92EF92FF920F931F93CF93DF93FF
:1025D00000D000D000D0CDB7DEB70E94E2040DE0FD
:1025E00010E0AA24A394B12C902E802F0E94D00535
:1025F000980127583E4F6901F901F080F826A1F4AF
:102600000150110988F78FEF89838A831B820E940A
:10261000371E8160782F9D838C8349815A816B811D
:102620008D810E9474132FC09091DC0191FF04C032
:102630008E830E94D6058E8125E030E0A501022E12
:1026400001C0440F0A94EAF7E42E4F21C1F0298318
:102650009A828E2191E009F490E09B830E94371EBC
:102660008160782F9D838C8349815A816B818D8114
:102670000E947413F6018081E826E08204C0215094
:102680003109E0F6BDCF0E94D721109178010E9458
:1026900086121817B9F00E94861280937801269648
:1026A0000FB6F894DEBF0FBECDBFDF91CF911F9163
:1026B0000F91FF90EF90DF90CF90BF90AF909F90E1
:1026C0000C947F0B26960FB6F894DEBF0FBECDBFDD
:1026D000DF91CF911F910F91FF90EF90DF90CF90FE
:1026E000BF90AF909F900895CF93DF93CDB7DEB7A3
:1026F0002B970FB6F894DEBF0FBECDBF4F83588720
:1027000069877A878B87DE01119686E0FD01119239
:102710008A95E9F785E0FE01379601900D928A953A
:10272000E1F749815A816B817C818D819E810E9474
:10273000BD192B960FB6F894DEBF0FBECDBFDF914B
:10274000CF910895CF93882309F4C2C0C82F82384F
:1027500059F40E94861281FDBBC089E30E94971C38
:102760000E94641D89E30CC0833879F40E948612AC
:1027700080FDAEC083E50E94971C0E94641D83E526
:102780000E94D91CCF910C94641D843859F40E9486
:10279000861282FD9DC087E40E94971C0E94641DE2
:1027A00087E4EECF8CEF8C0F813A48F48C2F0E9497
:1027B0001A2481118DC08C2F0E94971CE3CF80E2D8
:1027C0008C0F883048F4C77081E001C0880FCA952B
:1027D000EAF70E941D1DD6CF8BE58C0F833078F46D
:1027E000C53A29F0C63A31F083E890E005C081E8A7
:1027F00090E002C082E890E0CF910C94A81288E5A6
:102800008C0F833108F064C0C83A39F1C93A41F1FC
:10281000CA3A49F1CB3A51F1CC3A59F1CD3A61F18A
:10282000C03B69F1CE3A71F1CF3A79F1C13B81F108
:10283000C23B89F1C33B91F1C43B99F1C53BA1F186
:10284000C63BA9F1C73BB1F1C83BB9F1C93BC1F1E6
:10285000CA3BC9F180E090E038C082EE90E035C01C
:1028600089EE90E032C08AEE90E02FC085EB90E0D8
:102870002CC086EB90E029C087EB90E026C08CEC62
:1028800090E023C08DEC90E020C083E891E01DC073
:102890008AE891E01AC082E991E017C084E991E0EA
:1028A00014C081E292E011C083E292E00EC084E2A3
:1028B00092E00BC085E292E008C086E292E005C09B
:1028C00087E292E002C08AE292E0CF910C94BE12BD
:1028D000CF910895882309F44BC0823859F40E949F
:1028E000861281FF45C089E30E94971C0E94641DE7
:1028F00089E30CC0833871F40E94861280FF38C0CF
:1029000083E50E94971C0E94641D83E50E94D91CE8
:102910000C94641D843859F40E94861282FF28C0EA
:1029200087E40E94971C0E94641D87E4EFCF9CEF10
:10293000980F913A58F390E2980F983050F48770BE
:1029400091E001C0990F8A95EAF7892F0E94231D13
:10295000DFCF9BE5980F933020F480E090E00C945B
:10296000A812885A833120F480E090E00C94BE12C3
:102970000895882321F00E941D1D0C94641D089564
:10298000882321F00E94231D0C94641D08957F92DA
:102990008F929F92AF92BF92CF92DF92EF92FF926F
:1029A0000F931F93CF93DF931F92CDB7DEB77C01B8
:1029B000C62E772EFC01058102950F701281111130
:1029C0000E943A1D0E94901C882379F0112369F01F
:1029D00080E28C0D883048F082E00E94791C0E94D1
:1029E000901C91E0D82ED92601C0D12CE72DE2957C
:1029F000EF70F0E0E059FF4F0C944F26872D807F59
:102A0000072D0F70882311F00295007F112389F0A4
:102A1000002309F490C180E28C0D883020F4802FCF
:102A20000E941D1D03C0802F0E942D1D0E94641D49
:102A300082C18C2D0E946A14002309F495C180E2A2
:102A40008C0D883020F4802F0E94231D03C0802F1E
:102A50000E94331D0E94641D87C1972D907F872D92
:102A60008F70903211F08295807FCC2021F0F1E0C0
:102A7000CF16B1F01EC0112349F0002309F414C190
:102A8000013009F011C10E944D1D6EC1002319F0E3
:102A9000013009F469C189830E94501D89810AC1EE
:102AA000112321F0023008F05FC1FEC001115CC1AA
:102AB00001C1112321F0002309F4F6C03CC1002319
:102AC00009F4F8C03EC1872D86958695837090E005
:102AD000009719F0019761F047C1112321F08C2D67
:102AE000972D937002C080E090E00E94A8123CC134
:102AF000112321F08C2D972D937002C080E090E07F
:102B00000E94BE1231C18C2D112319F00E94DF20CA
:102B100002C00E9447210E94CC2126C1872D8370CC
:102B200009F052C0111120C18C2D829586958770B5
:102B3000880F880F9C2D9F70892E912CA12CB12C71
:102B4000082E04C0880C991CAA1CBB1C0A94D2F73E
:102B5000C4FE14C00FE010E020E030E0B901A8018D
:102B600004C0440F551F661F771F8A95D2F7CB010B
:102B7000BA01609570958095909503C060E070E013
:102B8000CB01272D26952695237030E02230310584
:102B900069F02330310589F0682979298A299B2930
:102BA0002130310571F00E94051BDEC068297929AA
:102BB0008A299B290E94211BD7C00E94051BC501A1
:102BC000B4010E94E91AD0C0112319F0872D817039
:102BD00001C08695882309F4C7C08C2D82958695FF
:102BE0008770880F880F9C2D9F70892E912CA12CA7
:102BF000B12C082E04C0880C991CAA1CBB1C0A947A
:102C0000D2F7C4FE14C00FE010E020E030E0B901BC
:102C1000A80104C0440F551F661F771F8A95D2F77D
:102C2000CB01BA01609570958095909503C060E0E6
:102C300070E0CB01272D269526952370422F50E07A
:102C40004230510569F04330510589F068297929EE
:102C50008A299B294130510571F00E94DF1B84C0F5
:102C6000682979298A299B290E94FB1B7DC00E9423
:102C7000DF1BC501B4010E94C31B76C08C2D90E000
:102C8000FC01E05EF109E531F10508F050C0E058C3
:102C9000FF4F0C944F260C2D0F70872D8F71112331
:102CA00031F00E945C1B802F0E94B9145DC00E940D
:102CB0007D1B802F0E94C01457C0112339F00111D1
:102CC00053C0872D8F710E94A21B4EC0023008F0A6
:102CD0004BC0F7CF112339F0872D8F710E945C1BF9
:102CE00043C01123C9F3872D8F710E947D1B3CC007
:102CF000112329F0872D8F710E94471B35C00E9438
:102D00003D1B32C0112351F0172D1F71812F0E94DE
:102D10005C1B63E0812F0E94701C26C081E00E9432
:102D2000791C023008F182E00E94791C1DC0112339
:102D300031F0002389F28C2D0E94A21315C00023CC
:102D400091F28C2D0E946A140FC0472D4F706C2D8C
:102D5000C7010E94AC060E94611A06C0472D4F7041
:102D60006C2DC7010E948E08DD20F9F00E946C1CBA
:102D700080FD1BC0F70112820E94661C0E945C1B32
:102D8000C7010E94E4160E94661C0F90DF91CF914C
:102D90001F910F91FF90EF90DF90CF90BF90AF9079
:102DA0009F908F907F900C947D1B0F90DF91CF911F
:102DB0001F910F91FF90EF90DF90CF90BF90AF9059
:102DC0009F908F907F9008950F931F93CF93DF93E1
:102DD000EC01888199812B813C81232BB9F09F3FA5
:102DE00011F48F3F99F0CE010E94E607882371F01D
:102DF000688179818A810E94621C8C010E94171C63
:102E00000E94DE1AB801CE010E94C714DF91CF9153
:102E10001F910F9108950E943A1D0E944A1D0E9421
:102E20000F1D0E94641D0E947D220E94CC2180E023
:102E300090E00E94A81280E090E00C94BE120E94E4
:102E40002A1D0C940B170E94571C292F22952F70B6
:102E500030E02C3031054CF42A3031056CF422502E
:102E6000310922303105A8F407C02C30310569F052
:102E70002F30310551F00DC0803F69F018F4803ECD
:102E800040F409C0843F29F406C093FB882780F9E9
:102E9000089580E0089581E00895CF93DF9300D0F6
:102EA00000D01F92CDB7DEB70F900F900F900F900C
:102EB0000F90DF91CF910895CF93DF9300D000D092
:102EC00000D0CDB7DEB726960FB6F894DEBF0FBEA2
:102ED000CDBFDF91CF9108951F93CF93DF93C09122
:102EE000870116E080918801C81799F0D0E01C9FF7
:102EF000F0011D9FF00D1124E757FE4F40815181D5
:102F000062817381848195810E945C172196C770CC
:102F1000E9CFDF91CF911F9108954091B901509170
:102F2000BA016091BB017091BC018091BD0190918B
:102F3000BE010C945C178091BE0182958F7009F0E0
:102F400054C08091BB01882309F44FC08091870150
:102F5000A09188016091B9017091BA014091BC01C2
:102F60005091BD01B6E08A1709F43FC090E04115C9
:102F70005105C1F17F3F11F46F3FA1F1B89FF001FE
:102F8000B99FF00D1124E757FE4F218172132AC01B
:102F90002081621327C02281211124C02381348122
:102FA0002417350710F421503109241B350B283C18
:102FB0003105C0F42091BE012F7020612093BE0125
:102FC00026E0289FF001299FF00D1124E257FE4FC3
:102FD00080818F708061808389EB91E00E94E4168C
:102FE0000C946C1701968770BECF0895CF92DF9234
:102FF000EF92FF920F931F93CF93DF93CDB7DEB77E
:1030000062970FB6F894DEBF0FBECDBF8C0185E08E
:10301000F801DE011D9601900D928A95E1F7D80125
:103020004C9111965C91119712966C911297139690
:10303000CD90DC9014973091B9017091BA018091D4
:10304000BC019091BD01009709F46BC17F3F19F459
:103050003F3F09F466C1E090BB01EE2009F4C0C017
:103060002091BE01C816D90628F0F601E81BF90B1D
:10307000CF0104C0809590958C0D9D1DFF24F39485
:10308000883C910578F0F12C207F09F0C6C07C2D9A
:10309000D98AC88A89890E944D1789EB91E00E94DC
:1030A000E416B1C0822F807F09F046C0751314C0AA
:1030B000341312C0611110C02F7020612093BE0123
:1030C0000E948D1789EB91E00E94E4168091BE0169
:1030D000D80115968C932EC0CD2819F15F3F11F4BD
:1030E0004F3FF9F0F62E61111CC0809187012091AD
:1030F000880136E0821709F45AC090E0389FF00149
:10310000399FF00D1124E757FE4F7181571306C008
:103110007081471303C07281711103C001968770DB
:10312000E9CFF62E662309F418C18091BE018160B3
:103130008093BE01F12C11C1751308C0341306C071
:10314000611104C08091BE01D801C3C04D875E8764
:103150008D859E856A8B0E9423176A898823E1F1F9
:103160006623D1F12091BE01822F82958F7090E06D
:10317000029774F08091B9019091BA0198878F837A
:103180001986DB86CA862C87CE0107960E94E41634
:1031900086E0F801A9EBB1E001900D928A95E1F784
:1031A0000E949B170E948D17FF24F394D6C04D8771
:1031B0005E878D859E850E94571C292F22952F7032
:1031C00030E0223031050CF0BCC09F7009F0B6C071
:1031D000805E883008F4C1C0C8010E94E416E4CFC4
:1031E000C816D90608F453C0F601E81BF90BCF0145
:1031F000883C910508F450C0F12C7C2DD98AC88AEE
:1032000089890E944D17E9EBF1E086E0DF011D920C
:103210008A95E9F70E948D17A0C0751314C0341366
:1032200012C0611110C08091BE01F8018583C801F0
:103230000E94E41686E0E9EBF1E0DF011D928A9539
:10324000E9F7FE2C8AC04D875E878D859E856A8B47
:103250000E9423176A89882309F4BECF662309F4E4
:10326000BBCF2091BE01822F82958F7090E0029794
:103270000CF48ECF8091B9019091BA019A83898321
:103280001B82DD82CC822E83CE0101967FCF80957A
:1032900090958C0D9D1DACCFF62E662309F49CCF26
:1032A00075132EC034132CC02091BE0120FD1FC009
:1032B000822F82958F70D9F0D80115962C9315978F
:1032C0008F3049F08F5F982F9295907F822F8F706B
:1032D000892B15968C93C8010E94E41686E0F801AC
:1032E000A9EBB1E001900D928A95E1F793CF86E0CA
:1032F000F801A9EBB1E001900D928A95E1F72DC09C
:103300004D875E878D859E850E942317811140CF52
:103310008091BE0181608093BE01C8010E94E416C5
:103320001CC0662309F458CF4D875E878D859E8526
:103330000E942317882309F44FCF2ACF811148CF49
:103340000CC0243031050CF047CF9F7009F440CFFA
:10335000F8019581907F09F03BCF8F2D62960FB6D3
:10336000F894DEBF0FBECDBFDF91CF911F910F91BB
:10337000FF90EF90DF90CF9008951F93CF93DF934E
:10338000CDB7DEB72C970FB6F894DEBF0FBECDBF1A
:103390004F83588769877A878B879C87CE010796EA
:1033A0000E94F617882369F08F8198852A853B85CE
:1033B000232BF1F19F3F09F063C08F3F09F060C0FC
:1033C00037C086E0FE013796DE01119601900D921E
:1033D0008A95E1F76F817885EA85FB85309741F121
:1033E0007F3F11F46F3F21F12091880130E0C90146
:1033F0000196877099274091870150E084179507BF
:1034000009F447C069837A83FD83EC8396E0929F39
:10341000D001939FB00D1124A757BE4FFE013196E6
:1034200001900D929A95E1F7809388010E946C17A4
:1034300016E080918701909188018917C1F1189F4A
:10344000C001112487579E4F0E94F617882379F1F7
:10345000E09187011E9FF0011124E757FE4F408144
:10346000518162817381848195810E945C17809172
:10347000870190E001968770992780938701D9CFC3
:103480004F81588569857A858B859C850E945C175C
:10349000CFCF0E941F171092880110928701E9EB8D
:1034A000F1E086E0DF011D928A95E9F7C1CF2C9605
:1034B0000FB6F894DEBF0FBECDBFDF91CF911F9145
:1034C0000895EF92FF920F931F93CF93DF938C0198
:1034D000009709F46CC0F12CEE24E394E8012196E6
:1034E000F8018491843740F4843008F051C0813071
:1034F00081F0823019F15BC0853709F444C0A8F12E
:103500009CE7980F903708F052C08F770E946A149A
:1035100041C00E5F1F4FFE01C49180E28C0F8830C6
:1035200048F4C7708E2D01C0880FCA95EAF70E9433
:103530003D1D14C08C2F0E94A2132DC00E5F1F4F83
:10354000FE01C49180E28C0F883058F4C7708E2D34
:1035500001C0880FCA95EAF70E94431D0E94641DAE
:103560001AC08C2F0E946A1416C00E5F1F4FFE01F6
:10357000C491CC2381F08FE99FE00197F1F700C05F
:103580000000C150F6CF0E5F1F4FFE01F49003C044
:103590000E94A2138E018F2D882309F49FCFEFE99B
:1035A000FFE03197F1F700C000008150F5CFDF91C7
:1035B000CF911F910F91FF90EF9008950895609320
:1035C000C3017093C4018093C5019093C6010C940C
:1035D0000B170F931F930091C3011091C401209109
:1035E000C5013091C601DC01CB01802B912BA22BB0
:1035F000B32B8093C3019093C401A093C501B093F2
:10360000C6011F910F910C940B170F931F930091FC
:10361000C3011091C4012091C5013091C601DC01A4
:10362000CB0180239123A223B3238093C3019093E2
:10363000C401A093C501B093C6011F910F910C94D2
:103640000B170F931F930091C3011091C401209198
:10365000C5013091C601DC01CB0180279127A2274B
:10366000B3278093C3019093C401A093C501B09385
:10367000C6011F910F910C940B171092BF0110926D
:10368000C0011092C1011092C2010C940B1741E0CD
:1036900050E060E070E004C0440F551F661F771FC4
:1036A0008A95D2F74093BF015093C0016093C10146
:1036B0007093C2010C940B1741E050E060E070E0A1
:1036C00004C0440F551F661F771F8A95D2F780915B
:1036D000BF019091C001A091C101B091C201482BDE
:1036E000592B6A2B7B2B4093BF015093C0016093F1
:1036F000C1017093C2010C940B1741E050E060E0EF
:1037000070E004C0440F551F661F771F8A95D2F7DB
:1037100040955095609570958091BF019091C00142
:10372000A091C101B091C201482359236A237B2390
:103730004093BF015093C0016093C1017093C201D7
:103740000C940B1741E050E060E070E004C0440FBF
:10375000551F661F771F8A95D2F78091BF01909100
:10376000C001A091C101B091C201482759276A2721
:103770007B274093BF015093C0016093C1017093B8
:10378000C2010C940B170F931F930091BF0110916E
:10379000C0012091C1013091C201DC01CB01802B1D
:1037A000912BA22BB32B8093BF019093C001A093C8
:1037B000C101B093C2011F910F910C940B170F938D
:1037C0001F930091BF011091C0012091C101309160
:1037D000C201DC01CB0180239123A223B323809378
:1037E000BF019093C001A093C101B093C2011F918A
:1037F0000F910C940B170F931F930091BF01109121
:10380000C0012091C1013091C201DC01CB018027B0
:103810009127A227B3278093BF019093C001A09363
:10382000C101B093C2011F910F910C940B17089521
:10383000CF92DF92EF92FF920F931F93CF93DF937C
:103840008C01C090C301D090C401E090C501F090FC
:10385000C6018091BF019091C001A091C101B091BA
:10386000C201C82AD92AEA2AFB2ACFE1D0E0D7012F
:10387000C6010C2E04C0B695A795979587950A9416
:10388000D2F780FF06C0B8018C2F0E94E40A01978E
:1038900021F4219760F780E001C08C2FDF91CF9158
:1038A0001F910F91FF90EF90DF90CF900895CF93ED
:1038B000DF93EC010E94181CBE010E94E40ADF9114
:1038C000CF910895CB010E94571C08958091C701A4
:1038D00085958595859508958091C7018770089590
:1038E00098E0899F90011124262B2093C7010C9406
:1038F0005C1B2091C701809582238093C701982F7C
:10390000977069F430E0482F552747FD50952417EC
:10391000350729F08595859585950C947D1B08952F
:103920009091C701977081E009F480E0089590912B
:103930000C01992321F090910D01911109C0209162
:103940000E0130910F01F90132969FEF40E01FC048
:10395000982F9695969596959F3050F5E0910E018B
:10396000F0910F01E90FF11D877021E030E0A9010E
:1039700002C0440F551F8A95E2F7CA019181892B35
:10398000818308959F3F39F04F5F4E3041F0519150
:103990005813F8CF0DC05111F7CF942FF5CF9F3F9B
:1039A00039F0F901E90FF11D97FDFA958283089529
:1039B000089590910C01992321F090910D0191119E
:1039C00009C020910E0130910F01F9013296205F5C
:1039D0003F4F1FC0982F9695969596959F30F0F47F
:1039E000E0910E01F0910F01E90FF11D877021E0C8
:1039F00030E0A90102C0440F551F8A95E2F7CA01C1
:103A0000809591818923818308953196E217F30788
:103A100029F090819813F9CF1082F7CF089581E0B3
:103A200090E0E0910E01F0910F01E80FF91F108274
:103A3000019680319105A9F708959091DB01892BBA
:103A40008093DB01089580959091DB018923809319
:103A5000DB0108951092DB0108959091DA01892B22
:103A60008093DA01089580959091DA0189238093FB
:103A7000DA0108951092DA0108959091D901892B05
:103A80008093D901089580959091D90189238093DD
:103A9000D90108951092D90108958093C80108951D
:103AA0001092C801089580910E0190910F01FC01C0
:103AB00031969C01205F3F4F80E0919191118F5F83
:103AC000E217F307D1F70895E0910E01F0910F018D
:103AD0008091DB018083E0910E01F0910F019081D4
:103AE0008091DA01892B8083E0910E01F0910F0122
:103AF00090818091D901892B80838091C80188238E
:103B000061F0E0910E01F0910F019081892B80838B
:103B10000E94531D81111092C80180910E01909155
:103B20000F010C94921220E0009739F0AC01415043
:103B30005109842395232F5FF7CF822F0895CF92C9
:103B4000DF92EF92FF926C01EE24FF24C114D104A6
:103B5000E104F10421F0C701B60120E101C020E039
:103B6000C72ED82EE92EFF24C114D104E104F1049C
:103B700019F0285FC701B6016B017C0154E0F6948F
:103B8000E794D794C7945A95D1F7C114D104E104AE
:103B9000F10419F02C5FC701B6016B017C0142E012
:103BA000F694E794D794C7944A95D1F7C114D104F9
:103BB000E104F10419F02E5FC701B601DC01CB016D
:103BC000B695A79597958795892B8A2B8B2B09F00E
:103BD0002F5F822FFF90EF90DF90CF90089580911C
:103BE000F301843021F11092DD0120E488E190E0BE
:103BF0000FB6F894A895809360000FBE20936000E4
:103C000080E00E947F0B83B7817F846083BF83B78E
:103C1000816083BF7894889583B78E7F83BF88E166
:103C20000FB6F89480936000109260000FBE089564
:103C3000089508950E94181E0E94E2040E94191E11
:103C40000E94D70591E0811101C090E0892F08956D
:103C50000E941F170E9486120C947F0B82E084BD85
:103C600093E095BD9AEF97BD80936E0008952FB7AE
:103C7000F8948091DE019091DF01A091E001B09174
:103C8000E1012FBF0895CF92DF92EF92FF920F9341
:103C90001F932FB7F8944091DE015091DF0160919E
:103CA000E0017091E1012FBF6A017B01EE24FF2446
:103CB0008C0120E030E0C016D106E206F30610F4D5
:103CC000415051099A01281B390BC9011F910F91CD
:103CD000FF90EF90DF90CF9008951F920F920FB654
:103CE0000F9211248F939F93AF93BF938091DE0126
:103CF0009091DF01A091E001B091E1010196A11D39
:103D0000B11D8093DE019093DF01A093E001B09399
:103D1000E101BF91AF919F918F910F900FBE0F90D6
:103D20001F9018950E94830FF8942FEF87EA91E671
:103D3000215080409040E1F700C0000087E090EB08
:103D4000DC018093FD019093FE01A093FF01B093ED
:103D500000029CE088E10FB6F894A895809360007B
:103D60000FBE90936000FFCFEF92FF920F931F93CF
:103D7000CF93DF93D82FCDE08C2F0E94D00505E0A4
:103D800010E0E82EF12CC701002E02C09595879512
:103D90000A94E2F780FF09C0602F7C2F80E00E9428
:103DA0008F08D81302C081E006C00150110958F7EE
:103DB000C15010F780E0DF91CF911F910F91FF90DC
:103DC000EF900895CF93C82F8CE20E94B41E8823F1
:103DD00021F08C2FCF910C94B41E80E0CF910895E8
:103DE000CF930E943720811102C00E941D20C5E69A
:103DF000C15049F00E94E2048FE39CE90197F1F77A
:103E000000C00000F5CF89E20E94E21E811113C1BB
:103E10008AE20E94E21E81110E941D2085E00E941C
:103E2000E21E81110E94921E0E9442208093DC01BA
:103E300087E00E94E21E8823A9F18BE10E94E21E26
:103E4000882351F08091DC0181FB222720F991E049
:103E5000922790FB81F90EC08EE00E94E21E88231B
:103E600061F08091DC0182FB222720F991E092270A
:103E700090FB82F98093DC0115C080E10E94E21E74
:103E80009091DC01882341F093FB222720F981E007
:103E9000822780FB93F904C0892F809580FB90F9DD
:103EA0009093DC018091DC010E9446200E94542006
:103EB0008093FC0180EE0E94E21E882341F08091F5
:103EC000FC01982F909590FB80F98093FC0189E389
:103ED0000E94E21E882359F08091FC0181FB222779
:103EE00020F991E0922790FB81F98093FC0182EE0A
:103EF0000E94E21E882359F08091FC0182FB222758
:103F000020F991E0922790FB82F98093FC0186EEE4
:103F10000E94E21E882359F08091FC0183FB222736
:103F200020F991E0922790FB83F98093FC0183EEC6
:103F30000E94E21E882359F08091FC0184FB222715
:103F400020F991E0922790FB84F98093FC0185E3AE
:103F50000E94E21E882359F08091FC0185FB2227F4
:103F600020F991E0922790FB85F98093FC0181E391
:103F70000E94E21E882359F08091FC0186FB2227D3
:103F800020F991E0922790FB86F98093FC0181E172
:103F90000E94E21E882359F08091FC0187FB2227B2
:103FA00020F991E0922790FB87F98093FC018091A2
:103FB000FC010E9458208091FC0187FB882780F932
:103FC00080930D0187E20E94E21EC82F8EE10E94BD
:103FD000E21E8111C2608FE10E94E21E8111C46065
:103FE00080E20E94E21E8111C86081E20E94E21E0E
:103FF0008111C06182E20E94E21E8111C06283E2EF
:104000000E94E21E8111C06484E20E94E21E8823A5
:1040100011F0C06802C0CC2329F08C2F0E944F20E1
:104020006C2F03C00E944B20682F70E080E090E06E
:10403000CF910C94DF1ACF9108956DEE7EEF80E062
:1040400090E00E94892660E082E090E00E9477265E
:1040500060E083E090E00E94772660E084E090E0FA
:104060000E94772660E085E090E00C94772680E05F
:1040700090E00E94712621E08D3E9E4F09F020E0E5
:10408000822F089582E090E00C946926682F82E0E8
:1040900090E00C94772683E090E00C946926682FDA
:1040A00083E090E00C94772684E090E00C946926FD
:1040B000682F84E090E00C9477268091E40180FFE3
:1040C0000BC06091130185E0689FB00111247595C4
:1040D0006795759567952BC081FF09C060911301A5
:1040E00085E0689FB00111247595679520C082FF17
:1040F00007C06091130185E0689FB001112417C0CB
:104100009091E5019923D1F060911201961788F7FB
:104110002091130185E0289F90011124929FA00116
:10412000939F500D112470E0CA010E943B26603815
:10413000710540F46115710539F002C065E070E069
:10414000862F08958FE7089581E008958091E40116
:1041500080FF08C06091110170E0759567957595B5
:10416000679521C081FF06C06091110170E07595CF
:10417000679519C082FF04C06091110170E010C002
:104180009091E5019923C1F0609110019617A0F775
:1041900080911101899FC001112470E00E943B268B
:1041A0006038710528F46115710521F0862F089596
:1041B0008FE7089581E0089561E070E0F4CF803FDB
:1041C00021F40E945D20819504C0813F29F40E9462
:1041D0005D208093E8010895823F21F40E945D20D4
:1041E000819504C0833F29F40E945D208093E701FC
:1041F0000895893F19F40E94A62005C08A3F31F432
:104200000E94A62081958093E90108958B3F21F4B7
:104210000E94A620819504C08C3F29F40E94A6200C
:104220008093EA010895843F21F48091E601816042
:1042300017C0853F21F48091E601826011C0863F5E
:1042400021F48091E60184600BC0873F21F48091C6
:10425000E601886005C0883F31F48091E601806105
:104260008093E60108958D3F21F48091E4018160FF
:104270000BC08E3F21F48091E401826005C08F3F26
:1042800029F48091E40184608093E4010895803FE3
:1042900039F48091E80187FF6CC01092E80169C091
:1042A000813F29F48091E8011816BCF362C0909117
:1042B000E701823F29F497FF5CC01092E70159C0E3
:1042C000833F19F41916CCF354C0893F41F480910F
:1042D000E90118160CF04DC01092E9014AC08A3F5E
:1042E00029F48091E90187FF44C0F6CF8B3F39F470
:1042F0008091EA0187FF3DC01092EA013AC08C3FED
:1043000029F48091EA011816BCF333C0843F21F4EC
:104310008091E6018E7F17C0853F21F48091E601F0
:104320008D7F11C0863F21F48091E6018B7F0BC009
:10433000873F21F48091E601877F05C0883F31F4F3
:104340008091E6018F7E8093E60113C08D3F21F4BA
:104350008091E4018E7F0BC08E3F21F48091E401B7
:104360008D7F05C08F3F29F48091E4018B7F80937E
:10437000E4018091E70181110EC08091E801811173
:104380000AC08091E901811106C08091EA01811182
:1043900002C01092E501089586EE91E00E949D1200
:1043A0000E94371E9093E3018093E20108951F93CA
:1043B000CF93DF938091E2019091E3010E94431E2D
:1043C000AC019091E501992321F02091140130E096
:1043D00006C0209115018AE0289F90011124421700
:1043E000530708F486C08091E701C091E801D0919D
:1043F000E9011091EA01811107C0C11176C0D11104
:1044000074C0111172C075C09F3F19F09F5F9093E7
:10441000E501181624F40E945D208093E701809145
:10442000E70187FF05C00E945D2081958093E70129
:104430001C1624F40E945D208093E8018091E8011D
:1044400087FF05C00E945D2081958093E8016091FF
:10445000E701662339F1C091E801CC2319F17727F0
:1044600067FD7095872F972F0E944C2523E333E338
:1044700043E35FE30E94B0250E9419256093E701A2
:104480006C2F772767FD7095872F972F0E944C25FB
:1044900023E333E343E35FE30E94B0250E94192541
:1044A0006093E8011D1624F40E94A6208093E90180
:1044B0008091E90187FF05C00E94A6208195809325
:1044C000E901111624F40E94A6208093EA0180914C
:1044D000EA0187FF05C00E94A62081958093EA012A
:1044E000DF91CF911F910C94CC219F3F09F08ECF8B
:1044F00096CFDF91CF911F910895E6EEF1E085E030
:10450000DF011D928A95E9F71092E5011092E4010E
:104510000895833081F128F4813059F08230D1F050
:104520000895853009F449C0B8F1863009F456C0C1
:10453000089580911501262F30E0280F311D2F3F5F
:10454000310524F4680F6093150108958FEF80936F
:104550001501089580911401262F30E0280F311D98
:104560002F3F310524F4680F6093140108958FEFF5
:1045700080931401089580911301262F30E0280FB5
:10458000311D2F3F310524F4680F60931301089506
:104590008FEF80931301089580911201262F30E050
:1045A000280F311D2F3F310524F4680F609312014D
:1045B00008958FEF80931201089580911101262FA5
:1045C00030E0280F311D2F3F310524F4680F609330
:1045D000110108958FEF80931101089580911001CA
:1045E000262F30E0280F311D2F3F310524F4680FAE
:1045F0006093100108958FEF809310010895833028
:1046000011F128F4813049F0823091F0089585301D
:1046100081F120F18630C1F108958091150168176C
:1046200020F4861B809315010895109215010895BA
:1046300080911401681720F4861B8093140108955B
:1046400010921401089580911301681720F4861BBD
:10465000809313010895109213010895809112011F
:10466000681720F4861B809312010895109212019E
:10467000089580911101681720F4861B8093110121
:10468000089510921101089580911001681720F487
:10469000861B8093100108951092100108950F93C6
:1046A0001F938D3109F46BC008F03FC08E3009F4C0
:1046B0007FC0C0F4873009F469C068F4863009F01F
:1046C000B1C08091DC01817F8E7F8093DC0181E02D
:1046D0008093EC01A8C0883009F4A2C08B3009F4A3
:1046E0009FC0A0C0863109F49BC078F4803109F4E2
:1046F00072C0813109F096C00E941F1790910D0180
:1047000081E0892780930D018BC0893109F488C02D
:104710008B3109F087C08091DC0181FB222720F9D1
:1047200091E0922790FB81F94CC0853309F470C069
:1047300048F4873209F46CC008F459C0893209F48E
:1047400067C070C0833438F48A3308F04EC08833B1
:1047500009F466C067C0833409F45AC0883409F08C
:1047600061C00E941F170FEF13ED20E301501040AE
:104770002040E1F700C000000E94921E51C00E943C
:10478000D3240E9486120E947F0B4AC09091DC01C4
:10479000892F8095817080FB90F929F09660986050
:1047A0009093DC0140C0997F977F9093DC0138C0E3
:1047B0008091DC0182FB222720F991E0922790FB77
:1047C00082F98093DC01992359F18091DC018160A9
:1047D0008093DC0125C08091DC0183FB222720F936
:1047E00091E0922790FB83F9ECCF895301C08D5162
:1047F00041E050E060E070E08A019B0104C0000FDE
:10480000111F221F331F8A95D2F7C901B80104C0B6
:1048100061E070E080E090E00E94DF1A0E941F17C4
:1048200081E001C080E01F910F91089580E008951C
:1048300080E00895CF93C82F8091EC01813079F00A
:1048400018F08230E9F187C0E0910E01F0910F017C
:104850008081813169F0823209F07FC009C0E09126
:104860000E01F0910F018081813111F0823261F4EB
:104870008C2F0E941624811104C08C2F0E944F237C
:104880001DC081E090E01AC08C2F0E941824811175
:1048900014C0C43179F048F4CB3079F0C03109F05C
:1048A00060C082E08093EC0108C0C93219F0C833BF
:1048B00021F057C01092EC0154C081E0817053C0C8
:1048C000C93289F118F5C43171F1A8F4C73009F083
:1048D00046C08AE08093150194E19093140193E01F
:1048E000909313018093120188E08093110188E274
:1048F0008093100134C0CE51C63088F5EC2FF0E023
:10490000E65DFE4F80818093EB0129C0CE34E9F053
:1049100020F4CB3421F56AE013C0C13579F0C235FB
:10492000F1F461E00DC08091EB01882319F0109241
:10493000EB0115C081E08093EC0115C061E006C079
:104940008091EB010E9489220AC06AE08091EB010C
:104950000E94FF2204C01092EC0180E004C081E0BC
:1049600002C080E0ABCFCF910895E1E8F0E0808114
:10497000886080838081816080838FB7F89493E022
:104980009093890090ED909388008FBF0895EFE693
:10499000F0E08081826080830895EFE6F0E080811E
:1049A0008D7F80830895EFE6F0E0908182E0892793
:1049B000808308951F920F920FB60F9211242F93A8
:1049C0003F934F935F936F937F938F939F93AF9397
:1049D000BF93EF93FF938091ED019091EE010196CB
:1049E0009093EE018093ED01811103C082E00E945B
:1049F0007F0BE091EE01E695E695F0E0EE51F84F81
:104A0000E4918091ED018E1303C080E00E947F0B42
:104A1000FF91EF91BF91AF919F918F917F916F9196
:104A20005F914F913F912F910F900FBE0F901F906C
:104A3000189504D06894B1118DC0089570D088F095
:104A40009F5790F0B92F9927B751A0F0D1F0660F7A
:104A5000771F881F991F1AF0BA95C9F712C0B13095
:104A600081F077D0B1E0089574C0672F782F882740
:104A7000B85F39F0B93FCCF3869577956795B395D4
:104A8000D9F73EF490958095709561957F4F8F4F43
:104A90009F4F0895E89409C097FB3EF49095809548
:104AA000709561957F4F8F4F9F4F9923A9F0F92FF4
:104AB00096E9BB279395F695879577956795B79572
:104AC000F111F8CFFAF4BB0F11F460FF1BC06F5F58
:104AD0007F4F8F4F9F4F16C0882311F096E911C06A
:104AE000772321F09EE8872F762F05C0662371F08B
:104AF00096E8862F70E060E02AF09A95660F771F9F
:104B0000881FDAF7880F9695879597F9089557FDCE
:104B10009058440F551F59F05F3F71F04795880F2B
:104B200097FB991F61F09F3F79F0879508951216C2
:104B300013061406551FF2CF4695F1DF08C016166E
:104B400017061806991FF1CF86957105610508941F
:104B50000895E894BB2766277727CB0197F9089536
:104B60000BD078C069D028F06ED018F0952309F0EA
:104B70005AC05FC01124EECFCADFA0F3959FD1F3D6
:104B8000950F50E0551F629FF001729FBB27F00DFB
:104B9000B11D639FAA27F00DB11DAA1F649F662750
:104BA000B00DA11D661F829F2227B00DA11D621F9F
:104BB000739FB00DA11D621F839FA00D611D221F59
:104BC000749F3327A00D611D231F849F600D211D3D
:104BD000822F762F6A2F11249F5750408AF0E1F0E0
:104BE00088234AF0EE0FFF1FBB1F661F771F881F29
:104BF00091505040A9F79E3F510570F014C0AACFC4
:104C00005F3FECF3983EDCF3869577956795B79513
:104C1000F795E7959F5FC1F7FE2B880F911D96953D
:104C2000879597F9089597F99F6780E870E060E0AD
:104C300008959FEF80EC089500240A941616170635
:104C400018060906089500240A941216130614067D
:104C500005060895092E0394000C11F4882352F0E0
:104C6000BB0F40F4BF2B11F460FF04C06F5F7F4F98
:104C70008F4F9F4F089597FB072E16F4009407D08F
:104C800077FD09D00E94552607FC05D03EF490958B
:104C900081959F4F0895709561957F4F0895EE0F10
:104CA000FF1F0590F491E02D0994AA1BBB1B51E155
:104CB00007C0AA1FBB1FA617B70710F0A61BB70B8C
:104CC000881F991F5A95A9F780959095BC01CD0131
:104CD0000895F999FECF92BD81BDF89A992780B5C4
:104CE0000895A8E1B0E042E050E00C949126262F10
:104CF000F999FECF92BD81BDF89A019700B40216D2
:104D000039F01FBA20BD0FB6F894FA9AF99A0FBE7F
:104D100008950196272F0E9478260C947726DC01AF
:104D2000CB01FC01F999FECF06C0F2BDE1BDF89AB6
:104D3000319600B40D9241505040B8F70895F89460
:024D4000FFCFA3
:104D42000220810B0F0CEC0BB80B840B0101C90183
:104D520028080A03140A3F4D3639A30756072007CD
:104D6200E7067A069306AC06C506010203040506A9
:044D72000708090025
:00000001FF
